:03000000020058A3
:03000B000204AB41
:100030002843292041647269616E20476F647769A3
:100040006E2031393937202D2061676F6477696EF2
:10005000406965652E6F726775810F12048E1204F8
:100060002CD2AF12086F020842752A00752B00755A
:100070002906752840752C0D752D23752E26753093
:100080007E752F317532578000753500753300E568
:1000900032B457028021B45302416BB45205753219
:1000A00053802EB44902801CB447028013B443022B
:1000B000801075325780007135BC00CD8D3280C9FB
:1000C00080C780C53198317D7D5931FA75325780AE
:1000D000B87533007E05E532DE027441B444028017
:1000E00054B446028016B45A028060B45302807C35
:1000F000B442028068B44102801C808D7532427126
:10010000DB40117D46AB3431FA7135513C71FD91C4
:100110000875324180C0E5316016753C22753D227C
:10012000753E42753F387B047D4131FA7135513C53
:1001300075324480A17D44AB3431FA7135513C9124
:1001400008753244500375325A808B7D5A7B0031DA
:10015000FA7135513C12040775324601D67D427B57
:100160000031FA7135513C75320001D6317D7D5335
:1001700031FA71355145319875324601D6783C7B5C
:100180000BEB83F6080BBB15F8EB24F5FB2262257D
:1001900020402D234E314E28783CE624E0F5F094A3
:1001A00040400375F04085F02808E624E1F5290871
:1001B000E624E0F52A08E66440F52B08E624E0F59D
:1001C0002C08E6F52D752E00752F31753000753130
:1001D00000EB24FBFB08DB02801FE6F52E08DB02A8
:1001E000801708DB028012E6F53008DB02800AE6A1
:1001F00024E0540860037531FF22E52BA82A08800B
:10020000025137D8FC740151377A00EB242351375F
:10021000E53324205137ED5137783C8005E65137DE
:10022000081BBB00F8EA33333354032A543F24201D
:100230005137E52C513722CA2ACA8154BD4E067463
:100240003F1C5C8004BD590EECB5330AE533045401
:100250003FF5337E05227DFF15811581BD540201D6
:10026000D6BDFF0201D675324101D67533007E0539
:10027000E532DE027441B44402802BB4460280664B
:10028000B452028007B45302800C01897135ECB579
:1002900033DE8D3280DA3198317D7D5931FA753215
:1002A0004675330180CA7135BD540280C3ECB53345
:1002B00015BD440712042240288069BD5A08120463
:1002C00007753246805EBD4102805B743F15335531
:1002D00033F533ECB5330ABD46028048BD44028095
:1002E00043753241808A7135BD54028083ECB53349
:1002F00015BD460A12040240267532448026BD42CE
:1003000005753200801E743F15335533F533ECB557
:10031000330DBD53057532534170BD5A02800575CA
:10032000324141707B007D5931FAE53304543FF589
:10033000337E054170E529F527E527B401037D5497
:10034000229144B401F3783C7A00717A24DEFB7187
:100350007A24E0FC717AFD8004717AF608DBFA7188
:100360007ACA9AFB33333354032B543F24E09A70F8
:10037000047DFF783C74C428FB22B87C06158115E7
:100380008180B212044450061581158180ABB401FE
:10039000061581158180AFCA2ACA22F5F0547FB5AF
:1003A0002D07A62D08E5F08014B47F02800824E014
:1003B0005004E5F08007A62D08744065F0F6087437
:1003C0003725289822E4B6230B081BE6547F6423C4
:1003D000600274406608C3DB01D322783C7913E9DC
:1003E00083F6080970F9E924ECF534E5350535C3E1
:1003F0006001B3225465737446696C6500902000F7
:10040000C322902000C32222783CE583335001228E
:10041000E0A3719B4005E5833350F5E824C4F5342F
:10042000C322783C71C5F0A350FAC322758DFD75C7
:100430008BFF53890F438920438840759850438729
:1004400080D29922209807E527B401F8D322C298D8
:10045000E599C3223099FDC299F59922C0E0C49173
:1004600066D0E0916622540F24028380E730313257
:1004700033343536373839414243444546740D915B
:1004800054740A9154229154A3E49370F922758C08
:1004900000758A005389F0438901D28C75246475F4
:1004A000260175250A752701D2A922758A6F758CD8
:1004B000FCD28CD52603752601D5240F752464D56E
:1004C000250975250AD527037527013204F526E588
:0E04D00026B401FB2224F6C31304D5E0FD225E
:1008000031300031300041565220412E4700540112
:10081000CE7401B25301F35601F87601FD70210543
:100820007801A17901A16D01DF00E520607BE52160
:10083000B45005900A818025B45305900908801DA5
:100840008067114B60FC12045480F775270A12046C
:100850004440F8F5F090080EB41B02E422E493B58E
:10086000F00675270574017360F8A3A3A380EE75E5
:1008700020007521508000C2B3D2B4D2B5740212E8
:1008800004CCC2A2759000C2B2C2A0C2A1C2A3C2CF
:10089000A4C295C296C297D2B774021204CC740D4A
:1008A000221204444003740D221177743F22121364
:1008B00038009008AE1204897400120454E422F542
:1008C000F09008ADA3E493D36003B5F0F722752050
:1008D0000012044440D311BF40CFF520740D221202
:1008E000044440C5F5F012044440BEB5F0BBF52108
:1008F000740D229008068008900800800390080379
:10090000120489E422E521225021B54C01774121CE
:100910003463214F43214B52216B442145642165AF
:100920006521A26C21886601A94601A973411E00B8
:10093000213201A912044440F9F52212044440F284
:10094000F523740D227AC07B0080087A4880027AF1
:1009500040AB22AC2312044440D8FD51337404123E
:1009600004CC740D227AA07B0080117A28AB22ACD3
:10097000237D0051331204547A20AB22AC237D0036
:1009800051331204547400227AAC12044440A3542C
:100990000644E0FB7C007D00513374041204CC74E7
:1009A0000D22D2B57AAC7B807C007D005133740A75
:1009B0001204CC801E11777590FFD2A2D2B2D2A0C1
:1009C000D2A1D2A3D2A4C2B3C297D296C2B77402A4
:1009D0001204CCC2B474641204CCD2B474161204DF
:1009E000CC7E208024DE0201A9D297D2B3C2B3D23A
:1009F000B3C2B3D2B3C2B3D2B3C2B3D2B3C2B3C21F
:100A000097D2B3C2B3D2B3C2B37AAC7B537C007D6E
:100A1000005133E520B43803BC53CA740D22780367
:100A2000187A307B00E8FC7D005133120454B80082
:100A3000EFE42279048AF0EBFAECFBEDFCE5F075CB
:100A4000F008D2B3C2B3D2B3C2B3339295A296D256
:100A5000B3C2B3D2B3C2B3D29700D2B3C2B3D2B38C
:100A6000C2B3D2B3C2B3D2B3C2B3D2B3C2B3C297CA
:100A700000D2B3C2B3D2B3C2B3D5F0C633FDD9B539
:100A8000225061A24C01774141BE6341CF4341E214
:100A900052612E4441F564614F6541AD6C611B6646
:100AA000610846616473617B0041AB01A974807188
:100AB000EDC2A100D2A1740F1204CC740D22120455
:100AC0004440E8F5F012044440E19109740D22120B
:100AD000044440D7F5F0741071EDE5F071FBC2A24B
:100AE00061D412044440C4F5F0741071EDE5F07166
:100AF000FBD2A261D412044440B1F5F0741171ED3F
:100B0000E5F071FBC2A261D4120444409E5421F569
:100B1000F0744071EDE5F071FB61C5120444408B47
:100B20005406F5F0742071EDE5F071FB61D47402A8
:100B300071ED7590FFD2A2C2A000E590D2A0120480
:100B400054C2A2C2A000E590D2A0120454E42274C0
:100B50000371ED7590FFC2A2C2A000E590D2A01271
:100B60000454E422740471ED7590FFD2A2C2A00077
:100B7000E590D2A0120454C2A2E422740871ED7868
:100B800003C2A218C2A4C2A38890D2B300C2B30009
:100B90007590FFC2A000E590D2A0120454B800E303
:100BA000E422D2B5D2B4C2B3C2B7C2A27590FFD20A
:100BB000B2D2A0D2A1D2A3D2A474021204CCC2B5E4
:100BC000C2B4740D22C2A175F00F74641204D5D59D
:100BD000F0F88003C2A100D2A175F0640030B20326
:100BE000740D2274641204D5D5F0F141ABD2A4C2C5
:100BF000A3C2A2F590D2B300C2B322C2A4D2A3C2B0
:100C0000A2F590D2B300C2B322C2A4C2A3C2A2F57D
:100C100090D2B300C2B3D2A285F090D2B300C2B3D7
:010C200022B1
:00000001FF
